:100000000C948300189518951895189518951895BF
:100010001895189518951895189518951895189578
:100020001895189518951895189518951895189568
:100030001895189518951895189518951895189558
:100040001895189518951895189518951895189548
:100050001895189518951895189518951895189538
:100060001895189518951895189518951895189528
:100070001895189518951895189518951895189518
:10008000189518951895189518951895392F482F83
:10009000F894E0E0F0E006C001968A352AE0920785
:1000A000D8F33196E017F10718F480E090E0F5CF2F
:1000B0007894842F932F0895BA93AA939A938A934E
:1000C0008EEF90E0AFE7B0E00FEF07BB08BB03C0D7
:1000D0008EEF90E0AFE7082F1A2F102318BB04E62D
:1000E00010E0D4DF8F3700E0900791F3AE3FB00708
:1000F00079F3880F991F8160B695A795A160EBCF22
:1001000000008895FECF0FE30DBF01E00EBFC0E2F7
:10011000D1E00E9491000E945C000E9480000C943B
:06012000800001E00895DB
:00000001FF
